:100000000C9433010C9450010C9450010C94500149
:100010000C9450010C9450010C9450010C9450011C
:100020000C9450010C9450010C9450010C9450010C
:100030000C9450010C9450010C9450010C945001FC
:100040000C9450010C9450010C9450010C945001EC
:100050000C94500130302C4F4B0032312C52454122
:1000600044204552524F520032362C575249544583
:100070002050524F54454354204F4E0033332C539D
:10008000594E544158204552524F520036322C4658
:10009000494C45204E4F5420464F554E4400363370
:1000A0002C46494C45204558495354530037332C6E
:1000B0004D4D433249454320444F532056302E384E
:1000C0000037342C4452495645204E4F5420524557
:1000D0004144590054005A0068007C008C009E0086
:1000E000AD00C1002C30302C3030004552524F5200
:1000F0003A2053442F4D4D43004552524F523A201F
:1001000046494C452053595354454D0046415431BE
:1001100036204F4B004641543332204F4B0045525E
:10012000524F523A2046494C4520464F524D415479
:1001300000203C4449523E000000004B04FD0735BE
:10014000077D1429072A11130B0B1073144436343E
:100150001719E1194E04E41A51045E1BF7184804FC
:1001600008194D32493622651EFE217F204020EAC3
:100170001DDF1DD21DC81D543634D71B9E1C4E04D6
:10018000201D51045B1C871B48049C1B50303054BD
:100190000400004E044B0451042A11130B4804754B
:1001A0000415151515151515151515151515151510
:1001B0001515131313131313131212121212121113
:1001C00011111111111111111144454C5345515088
:1001D000524755535252454C3F3F3F00424C4F43CC
:1001E0004B5320465245452E004552524F523A201D
:1001F000443634005441504520454E442E004D3283
:10020000492046494C45204552524F5200505247D2
:100210000044454C00204D3249002E4D324900002B
:100220002E50524700001E15112976140E16252453
:100230001B1A591C1D26362C2B2122232D2E3E3C09
:1002400033322A34353D4544423A313B43464EE948
:10025000FF49414B4D79ECFA55124A4C7CFD830322
:100260000405F2F45A6611241FBECFE5D8E0DEBFC4
:10027000CDBF10E0A0E6B0E0ECE7F9E402C00590E5
:100280000D92A43CB107D9F715E0A4ECB0E001C091
:100290001D92A23AB107E1F70E9452010C94BD24CD
:1002A0000C9400000E94820278940E941A0A0E9414
:1002B000FE230E94BB090E946D180E9498040E94B0
:1002C000A1220E945706FBCFBF92CF92DF92EF92FE
:1002D000FF920F931F93CF93DF937C0130E020E0D8
:1002E00000E010E0C0E6D0E0EEE2CE2E90E2D92EA3
:1002F00080E3B82E0FC0222309F450C0F701E30FAA
:10030000F11DB0820F5F1F4F24960A30110509F4CA
:100310004AC03F5F0130A1F1043091F1073081F113
:1003200088819981AA81BB81481759076A077B0791
:1003300010F3F701E30FF11D20E3208388819981F9
:10034000AA81BB81481759076A077B0788F0822F6B
:100350008F5F282F808388819981AA81BB81481B68
:10036000590B6A0B7B0B481759076A077B0778F70D
:1003700021E00F5F1F4F24960A30110551F613C07C
:10038000222331F0F701E30FF11DC0823F5FC8CF98
:10039000F701E30FF11DD0823F5FC2CFF701E30FFA
:1003A000F11DD082AFCFDF91CF911F910F91FF90C0
:1003B000EF90DF90CF90BF900895EF92FF920F9350
:1003C0001F93CF93DF937C0104E710E09B01442748
:1003D0005527E0E3D701EC93E80188819981AA8150
:1003E000BB81281739074A075B07A0F08E2F8F5F64
:1003F000E82FE7018883E80188819981AA81BB8180
:10040000681B790B9B0144275527281739074A0792
:100410005B0760F70894E11CF11C0C5F1F4FE0E0E4
:1004200008381E07B1F6DF91CF911F910F91FF9011
:10043000EF900895CF92DF92EF92FF920F931F9368
:10044000CF93DF93EC01E881E03271F5CC24C394C3
:10045000FE01EC0DF11D80818032C9F3D82E80534E
:100460008A3040F5EE24FF2487012AE030E040E0A6
:1004700050E0C801B7010E9470247B018C018D2DD2
:100480009927C097AA2797FDA095BA2FE80EF91EC5
:100490000A1F1B1FC394FE01EC0DF11DD0808D2D92
:1004A00080538A3030F309C0CC248E2FD82E80534D
:1004B0008A30C0F2EE24FF248701C801B701DF9122
:1004C000CF911F910F91FF90EF90DF90CF90089503
:1004D000009731F0ACE6B7E01197F1F70197D1F74B
:1004E000089526EE31E0482F9927249F812D349FCF
:1004F000800D911D112406971816190614F4019702
:10050000F1F7089582B3837E82BB81B3837E81BB82
:100510001092CF0088E08093D00008958A988B983D
:1005200084E60E94710281E090E008950F931F938A
:10053000CF93DF93082F162FC0E0D0E080B3802345
:10054000112329F090E0882309F491E0892F882372
:1005500091F482E00E94710221968DEFC83ED80787
:1005600069F78B988A9884E08093CF00849BFECFB4
:1005700081E090E002C080E090E0DF91CF911F9198
:100580000F9108958A9A86E40E9471028B9886E4FE
:100590000E94710261E088E00E94960290E0811161
:1005A00091E081E09827892F9927089560E088E0FD
:1005B0000E949602882319F080E090E008958A98BE
:1005C00086E40E9471028B9A86E40E94710281E0A7
:1005D00090E008950F931F93082F162F61E084E099
:1005E0000E949602882319F080E090E045C08B9825
:1005F00060E084E00E9496028823B1F7112339F568
:1006000084E10E94710210E00CC08A9886E40E9486
:1006100071028B9886E40E9471021F5F183031F0DE
:1006200006958B9A00FDF1CF8A9AF0CF8B9A8A9823
:1006300084E10E94710261E084E00E94960290E0F1
:100640008823A9F481E09827892F992715C088EC81
:100650000E94710261E084E00E949602882321F6E4
:1006600060E084E00E949602882351F2BDCF91E0C1
:1006700081E09827892F99271F910F91089561E0B4
:100680000E94EA02882319F480E090E008950E9415
:10069000C20220E030E0882311F021E030E0C901FF
:1006A000089560E00E94EA0299270895FF920F934F
:1006B0001F931092CF0060E088E00E94960288238A
:1006C000D9F58A98839B1CC010E002C0143141F018
:1006D0008AE00E9471021F5F8399F8CF143180F085
:1006E0008091CF0081608093CF008A9A86E40E9437
:1006F00071028A9861E088E00E9496028823E1F402
:10070000849B1DC010E000E00DC080E8F82E61E081
:1007100088E00E949602882379F416951F290F5FBE
:10072000083099F060E088E00E949602882321F466
:100730008299EBCFFF24EBCF80E090E009C080915D
:10074000CF0082608093CF00DDCF8A9A812F9927D6
:100750001F910F91FF9008950E94560399270895C5
:10076000CF92DF92FF920F931F93CF93DF936C0191
:10077000849974C08A9A8B9882E30E9471020E94C5
:100780005603982F8091CF0082FD32C08091D00017
:100790008062981781F50E945603982F8091CF00B0
:1007A00082FD26C0F6019083892F807F803609F470
:1007B0004CC09F3309F45FC000E010E0E60107C0C1
:1007C0000F5F1F4F21960932110591F09883F02E8B
:1007D0000E945603982F8091CF0082FD09C080911E
:1007E000CF0081FFEDCF9F3359F7C1E0D0E030C09B
:1007F000C4E0D0E044C08091D00080649817A1F597
:100800000E945603982F8091CF0082FDF1CFF60110
:100810009083FF2411C0839B0FC00E945603982F22
:100820008091CF0082FDE4CFF7E2FF1508F3F601D7
:10083000EF0DF11D9183F394849BEDCF0E94D602BE
:100840008823B1F2C3E0D0E003C0FF24C2E0D0E0CF
:1008500084E60E947102F601F1A611C08A988B9875
:10086000FF24C0E0D0E0F4CF84E60E9471028A98B1
:100870008B98849BFECFFF24C0E0D0E0E9CFCE016F
:10088000DF91CF911F910F91FF90DF90CF9008954E
:1008900081E090E0089581E090E0089582E090E0AA
:1008A000089580E090E008951F930E942A118334F8
:1008B00019F080E090E017C00E942A118633C9F732
:1008C0000E942A118433A9F710E00E942A111F5FA9
:1008D0001731D9F70E94130B20E030E0882311F480
:1008E00021E030E0C9011F9108951092D1000E94CB
:1008F000731481E090E008951092D3008FEF8093FD
:10090000D10086E08093D2000E94BB09882359F46D
:100910000E94570B80FF06C08091C400882311F00D
:100920001092D10008950E94370B0E946D18F0CFED
:100930000E947C049098889A84E190E00E9468026A
:10094000909A0895CF93DF93EC010E94AC03FE01CF
:1009500009958091CF0080FD04C08091CF0082FF77
:10096000F4CFDF91CF910895FF920F931F93CF9310
:10097000DF938C01F62EEA018091FC009091FD003E
:100980000596860F911D9093FD008093FC00809149
:10099000FC009091FD000E9451038091FC00909119
:1009A000FD00892F99270E945103802F0E94510337
:1009B000012F110F110B802F0E945103FF2051F0C6
:1009C00000E0FE01E00FF11D80810E9451030F5FE6
:1009D000F016B9F780E00E945103DF91CF911F918B
:1009E0000F91FF900895EF92FF921F93CF93DF93A3
:1009F0007C01EB01FC010995182F08C0812F0E9492
:100A00005103882339F0F7010995182FFE01099544
:100A10008823A1F3812F0E943F03DF91CF911F9183
:100A2000FF90EF9008950F931F938C0181E098E061
:100A30009093FD008093FC0081E00E94510388E0C8
:100A40000E94510384EB94E0F801099580E00E9434
:100A5000510380E00E943F031F910F9108950F936F
:100A60001F93CF93DF93E091D200FF27EE0FFF1F7C
:100A7000EC52FF4F25913491F9018491882349F07C
:100A8000E90121960E945103FE0121968491882359
:100A9000C9F7C4EED0E08E010B5F1F4FFE018491B9
:100AA0000E9451032196F0E0C93EDF07B9F7F80133
:100AB00084910E943F03DF91CF911F910F91089580
:100AC0000F931F93CF93DF938091FF00803451F1F8
:100AD00010E000E0CFEFD0E06AE370E0CE010E94CA
:100AE0002C24009719F0182F1C1B1F5F1123E9F00D
:100AF00040912701411790F0212F3327912FE92FA3
:100B0000FF27DF01A21BB30BA250BF4FE250FF4FE4
:100B10008181FD0181839F5F491788F7411B4093C5
:100B2000270103C011E001E0D5CF802F9927DF9185
:100B3000CF911F910F910895FF920F931F93CF9321
:100B4000DF93EC011092D3008091FF008F3559F0B4
:100B50008091C400882391F487E08093D2008FEFC6
:100B60008093D10098C0809100018F3589F78FEF75
:100B70008093D10081E08093D3008DC00E94570BF9
:100B800080FFEACF8091FF00843299F08F3541F0E9
:100B90000E946005882389F085E08093D3007BC0A4
:100BA0008091D100882301F18F3F09F474C0109225
:100BB000D10083E08093D3006EC08091D100882360
:100BC00009F041C0209127012223A9F090E03EE7DF
:100BD000EEEFF0E004C09F5F3196921760F48181E0
:100BE0008F3FC9F73183F7CF88E890E00E949215D4
:100BF0008823F9F650C08FEF90E00E949215882369
:100C0000C1F68FEF90E00E947D14882341F180911E
:100C10002701C82FDD27C450DF4F0DE411E041E06C
:100C2000F42E43E050E0B801CE010E940F24892B3E
:100C3000D1F0F3940B5E1F4F85E0F81691F782E038
:100C40008093D30028C08F3F31F1FE013996259162
:100C500034918FEF90E0F9010995882381F784E0C2
:100C60008093D20018C0F8013396259134918FEF0C
:100C700090E0F9010995882349F0F092D100F8013C
:100C8000359685919491892BD1F293CF1092D10012
:100C900084E08093D3006FEF70E084ED90E00E94D9
:100CA0003724DF91CF911F910F91FF900895CF933B
:100CB000DF9388E08093D0008EEF90E00E94B00335
:100CC000282F843009F4C2C0882309F4BFC090984B
:100CD000E091D100EF3FF1F085E1E89FE0011124C0
:100CE000C85CDE4FE0912701FF27E250FF4F1182E1
:100CF0008091FE00382F3F709927807F9070803E52
:100D0000910529F1803F910561F18036910529F027
:100D1000909A9CC0C0E0D0E0E5CF233009F441C0F8
:100D20002230B1F72097A1F18091D300853009F4EA
:100D300056C08091D200843009F451C085E0809380
:100D4000D20088E494E00E94A204909A7FC0209789
:100D5000F9F2FE01739685919491FC010995909AA0
:100D600075C03F3071F42097B9F0FE013796259198
:100D700034918FEF90E0F90109958093D200909A19
:100D800065C01092D200CE010E949C05909A5EC070
:100D900088E494E00E94A20487E08093D200909AB5
:100DA00055C03F3051F18091D300813061F18430E2
:100DB00091F1882381F0209771F0823009F43BC0D3
:100DC000833009F0A5CFFE013596859194910E945C
:100DD0001305909A3BC00E948E02909A37C0FE0184
:100DE0003B962591349184ED90E0F9010995882393
:100DF000C1F482E08093D200A4CF0E942F0510920C
:100E0000D200909A23C00E947C0483EA97E00E945B
:100E10001305909A1BC087E797E00E941305909AEC
:100E200015C01092D200FE017196859194910E9496
:100E3000A204909A0BC0FE013F9665917491FE0149
:100E40003D96859194910E94F304909ADF91CF9101
:100E500008950F931F938C010E94C714C8010E942C
:100E60006C1699271F910F9108951F93CF93DF93CD
:100E70001091FF006AE370E08FEF90E00E942C2455
:100E80000097D1F0EC012196133521F1123529F0AC
:100E90001E34A9F083E090E026C06DE370E0CE013F
:100EA0000E942C24FC01892B39F01192BE01CF0144
:100EB0000E944215882399F080E090E014C0CE0192
:100EC0000E947521882371F482E08093D10080E034
:100ED00090E009C0CE010E94C714882369F784E01E
:100EE00090E001C09927DF91CF911F910895EF9273
:100EF000FF920F931F93CF93DF93CDB7DEB7639726
:100F00000FB6F894DEBF0FBECDBF7C0142E150E0CA
:100F10006EE171E08E010F5F1F4FC8010E941C241B
:100F2000A80162E180E090E0F701099563960FB6B1
:100F3000F894DEBF0FBECDBFDF91CF911F910F910F
:100F4000FF90EF900895EF92FF920F931F93CF932E
:100F5000DF93CDB7DEB763970FB6F894DEBF0FBE51
:100F6000CDBF8C010E94570B982F8091C40088231D
:100F700001F1892F992780FF0FC082FF27C048E029
:100F800050E065E171E07E010894E11CF11CC701AD
:100F90000E941C2468E01FC042E150E069EF70E04D
:100FA0007E010894E11CF11CC7010E941C2462E12F
:100FB00012C04DE050E06BEE70E07E010894E11C41
:100FC000F11CC7010E941C246DE005C048E050E000
:100FD0006CE071E0D8CFA70180E090E0F8010995BE
:100FE00063960FB6F894DEBF0FBECDBFDF91CF91F1
:100FF0001F910F91FF90EF9008959F92AF92BF9233
:10100000CF92DF92EF92FF920F931F93CF93DF93D4
:10101000CDB7DEB76E970FB6F894DEBF0FBECDBF6B
:101020007C01E7E0AE2EB12CAC0EBD1E43E050E0DB
:1010300060E270E0C5010E94252482E28A870E9456
:101040007B0B6E010894C11CD11CA6010E947F0E6F
:10105000AC01009709F44FC0FC018081882309F49A
:101060004AC072E2972E853ED9F1FA0183858F300E
:10107000B9F1883009F47DC084FD58C0FA01848D2F
:10108000958DA68DB78D81509C4FAF4FBF4F6AE0B5
:10109000B695A795979587956A95D1F7F7E2803130
:1010A0009F07E0F195016EE00FE017E2DE011B966D
:1010B000FA0188E001900D928150E1F78EE28B8B6E
:1010C000DE015496FA01389683E001900D9281502A
:1010D000E1F79F8A2D5F3F4FA901C801F7010995EC
:1010E000C6010E947C12AC01892B29F0FA01808193
:1010F000882309F0B8CF8091C400882309F057C035
:101100004DE050E06BEE70E0C5010E941C24A5018B
:101110006DE080E090E0F701099549C063E0883E0A
:10112000960768F18C0195016EE0C0CFDE011B9639
:10113000FA0188E001900D928150E1F780E28B8BFB
:10114000DE015496FA01389683E001900D928150A9
:10115000E1F79F8A46E050E061E371E0CE014896F6
:101160000E941C24A50167E180E090E0F701099549
:10117000B7CF6BE080E090E0F7010995B1CF8436FE
:10118000910548F48A30910560F09E012B5F3F4F36
:101190008C0160E18BCF9E012A5F3F4F8C016FE095
:1011A00085CF9E012C5F3F4F8C0161E17FCF6E9612
:1011B0000FB6F894DEBF0FBECDBFDF91CF911F9168
:1011C0000F91FF90EF90DF90CF90BF90AF909F90E6
:1011D0000895CF93DF93CFEFDFEF03C0209731F077
:1011E00021978FEF0E942A0A8823C1F3CE01CD2BCD
:1011F00011F081E090E0DF91CF9108951F93CF939C
:10120000DF93182FCFEFDFE003C0209731F0219755
:101210008FEF0E942A0A8117C1F7CE01CD2B11F062
:1012200081E090E0DF91CF911F910895CF92DF92FE
:10123000EF92FF920F931F93CF93DF937B018C016B
:101240006A01C49888E50E942A0A89E0EE0CFF1C16
:10125000001F111F8A95D1F7C801B7010E94300AFB
:101260008FEF0E942A0A80E00E94FE08882331F452
:10127000C49A1092C40080E090E025C08EEF0E94D6
:101280002A0AC0E0D0E0F60181916F010E942A0A8B
:101290002196F2E0C030DF07B1F78FEF0E942A0AF3
:1012A0008FEF0E942A0A8FEF0E942A0A8F708530E2
:1012B000F9F60E94E9088823D9F2C49A8FEF0E94B8
:1012C0002A0A8FEF90E0DF91CF911F910F91FF904D
:1012D000EF90DF90CF900895CF92DF92EF92FF9240
:1012E0000F931F93CF93DF937B018C016A01C49806
:1012F00081E50E942A0A99E0EE0CFF1C001F111FD5
:101300009A95D1F7C801B7010E94300A8FEF0E9469
:101310002A0A80E00E94FE08882331F4C49A1092C1
:10132000C40080E090E01EC08EEF0E94FE0888237B
:10133000A9F3C0E0D0E08FEF0E942A0AF601819362
:101340006F012196F2E0C030DF07A9F78FEF0E940E
:101350002A0A8FEF0E942A0AC49A8FEF0E942A0A53
:101360008FEF90E0DF91CF911F910F91FF90EF9061
:10137000DF90CF9008951F931092C400C49A10E09C
:101380008FEF0E942A0A1F5F1A30D1F7C49880E4B9
:101390000E942A0A60E070E080E090E00E94300A3B
:1013A00085E90E942A0A81E00E94FE08882321F430
:1013B000C49A80E090E03CC0C49A8FEF0E942A0A51
:1013C000C4981FEF02C0112399F381E40E942A0AF6
:1013D00060E070E080E090E00E94300A8FEF0E94B1
:1013E0002A0A115080E00E94FE08882361F311232D
:1013F000F9F2C49A8FEF0E942A0AC49880E50E94ED
:101400002A0A60E072E080E090E00E94300A8FEFEC
:101410000E942A0A80E00E94FE08882349F2C49AAA
:101420008FEF0E942A0A8FEF8093C4008FEF90E025
:101430001F910895C79AC49ABF9ABE98BD9ABC9A44
:101440006C9A689869986B986A986D986E9A8EB144
:101450008FB108958FB9779BFECF8FB199270895EB
:101460009B01AC015FB9779BFECF8FB14FB9779BE2
:10147000FECF8FB13FB9779BFECF8FB12FB9779B4E
:10148000FECF8FB108958D9A959A8E9A969A089567
:1014900080FF03C0959A82B302C0959882B3969854
:1014A00086E2982F9A95F1F7969A8A95F1F7089522
:1014B000FF920F931F93182F80E00E94480A00E0CC
:1014C000FF24812F0E94480A812F8170F8261695EB
:1014D0000F5F0830B1F78F2D0E94480A81E00E940B
:1014E000480A8FE38A95F1F71F910F91FF900895B5
:1014F0008093C500807711F091980895919A08958E
:10150000611571058105910569F48091C50082FD21
:1015100024C0209163053091640540916505509188
:10152000660523C0625070408040904020912C0599
:1015300030912D05442755270E9470249B01AC0152
:1015400080915B0590915C05A0915D05B0915E0571
:10155000280F391F4A1F5B1F08C020915B0530917F
:101560005C0540915D0550915E05CA01B901089581
:1015700020915B0530915C0540915D0550915E05C1
:10158000621B730B840B950B20912C0530912D055C
:10159000442755270E949B242E5F3F4F4F4F5F4F9C
:1015A000CA01B90108959B01AC018091C50082FF79
:1015B00015C0220F331F441F551F232F342F452FD3
:1015C000552780915F0590916005A0916105B091CC
:1015D0006205280F391F4A1F5B1F10C0232F342FAD
:1015E000452F552780915F0590916005A091610579
:1015F000B0916205280F391F4A1F5B1FCA01B9014C
:1016000008958091C50083FF09C060914F057091D6
:1016100050058091510590915205089560E070E069
:1016200080E090E008958091C50083FF1DC060E0D8
:1016300070E020915705309158054091590550911F
:101640005A0580914F0590915005A0915105B09198
:101650005205281739074A075B0710F4CB01089594
:1016600061E070E0CB01089581E090E0089580E0B2
:101670000E94780A8FEF9FEFAFEFBFEF80932805AE
:1016800090932905A0932A05B0932B058093B3006E
:101690009093B400A093B500B093B6008093B700C8
:1016A0009093B800A093B900B093BA0008958091C8
:1016B000C50099270895609167057091680580912C
:1016C000690590916A05089580912C0590912D05EA
:1016D000089560912E0570912F05809130059091AD
:1016E0003105089560916F057091700580917105C5
:1016F0009091720508956091280570912905809157
:101700002A0590912B050895EF92FF920F931F9356
:10171000CF93DF93CDB7DEB72C970FB6F894DEBF2B
:101720000FBECDBF8C014CE050E0BC017E0108949F
:10173000E11CF11CC7010E944C2429812E32D1F1F9
:1017400080E090E0DE01129605C02D9101962E32C8
:1017500009F43FC0382F222309F448C0F801E80FEC
:10176000F91F20833F5F8730910579F7932FF701A9
:10177000E30FF11D80818E3251F19B3048F016C08D
:10178000F801E90FF11D80839F5F9B3079F03F5F87
:10179000F701E30FF11D8081882391F7F801E90F2C
:1017A000F11D80E280839F5F9B30C0F3C8010E94DF
:1017B000662420C08A818E32D9F091E0F801E90FC9
:1017C000F11D80E280839F5F9B30C0F313C03F5FB9
:1017D000D4CF932F3F5F983050F6F801E90FF11DF9
:1017E00080E280839F5F9830C1F7C1CF982FF3CFFD
:1017F00092E0E4CFF80113862C960FB6F894DEBF82
:101800000FBECDBFDF91CF911F910F91FF90EF9051
:1018100008959198899A84E190E00E946802919AD3
:1018200008958091C50086FF08954091AF005091C2
:10183000B0006091B7007091B8008091B9009091AC
:10184000BA000E941609882379F38091C5008F7B26
:101850000E94780A0895EF92FF920F931F937B01E5
:101860008C010E94110CE091AF00F091B00080E07B
:1018700092E011920197E9F7C801B7010E94800A2E
:101880006093B7007093B8008093B9009093BA004A
:1018900080912C0590912D05892BE9F010E0409165
:1018A000AF005091B0006091B7007091B800809186
:1018B000B9009091BA00610F711D811D911D0E94A8
:1018C00016091F5F212F332780912C0590912D053C
:1018D0002817390720F31F910F91FF90EF9008957B
:1018E000EF92FF920F931F937B018C018091B700C1
:1018F0009091B800A091B900B091BA008E159F05E3
:10190000A007B10751F00E94110CE092B700F092CD
:10191000B8000093B9001093BA001F910F91FF9087
:10192000EF900895DF92EF92FF920F931F938091B3
:10193000C50085FF38C0E090B300F090B40000917E
:10194000B5001091B6004091B1005091B200C801AD
:10195000B7010E941609882331F180913205823047
:10196000E8F071E0D72E8091670590916805A0910D
:101970006905B0916A05E80EF91E0A1F1B1F409108
:10198000B1005091B200C801B7010E941609882326
:1019900051F0D39480913205D81628F38091C50078
:1019A0008F7D0E94780A1F910F91FF90EF90DF903A
:1019B00008950E94160999270895AF92BF92CF9279
:1019C000DF92EF92FF920F931F93CF93DF937B01F0
:1019D0008C014091AF005091B0000E946C09809141
:1019E000AF009091B000EC012B9645E050E06BE821
:1019F00070E0C6960E943E24892B19F080E090E0AA
:101A00009BC08091C50081600E94780AAB80BC8039
:101A1000CC24DD24AE0CBF1CC01ED11E6D81862FD0
:101A20009927EB84FC848E9D90018F9D300D9E9DA7
:101A3000300D1124442755272A0D3B1D4C1D5D1DDB
:101A400020936305309364054093650550936605C4
:101A50008E819F81929582958F7089279F708927AB
:101A6000AA27BB27280F391F4A1F5B1F20935B053E
:101A700030935C0540935D0550935E050027112768
:101A8000E0926705F09268050093690510936A0576
:101A90008A81482F552750932D0540932C05A092FD
:101AA0005F05B0926005C0926105D09262056093B7
:101AB000320528853985C901AA27BB2780932E05C1
:101AC00090932F05A0933005B0933105232B61F43B
:101AD0008D899E89AF89B88D80932E0590932F05AF
:101AE000A0933005B0933105CA019C0144275527C6
:101AF00060912E0570912F058091300590913105F0
:101B00000E949B2420932E0530932F05409330058F
:101B10005093310510926F05109270051092710567
:101B200010927205109228051092290510922A052C
:101B300010922B0581E090E0DF91CF911F910F91E2
:101B4000FF90EF90DF90CF90BF90AF9008954F92AD
:101B50005F926F927F929F92AF92BF92CF92DF92ED
:101B6000EF92FF920F931F93CF93DF932B013C01D2
:101B70004091AF005091B0000E946C098091AF007D
:101B80009091B000EC012B9645E050E061E970E0E7
:101B90008E5A9F4F0E943E24892B19F080E090E0DE
:101BA00074C08091C50085600E94780AEB80FC803B
:101BB00000271127E40CF51C061D171D9D80692DBB
:101BC000772788279927A98CBA8CCB8CDC8CA60127
:101BD00095010E9470246E0D7F1D801F911F6093E0
:101BE0005B0570935C0580935D0590935E05A09204
:101BF0006705B0926805C0926905D0926A052A818E
:101C0000332730932D0520932C05E0925F05F09249
:101C10006005009361051093620590923205442798
:101C200055276D897E898F89988D0E949B242093EA
:101C30002E0530932F0540933005509331058DA12B
:101C40009EA1AA27BB27840D951DA61DB71D8093B5
:101C50006B0590936C05A0936D05B0936E0589A1FB
:101C60009AA1ABA1BCA180936F0590937005A0933E
:101C70007105B09372058093280590932905A09370
:101C80002A05B0932B0581E090E0DF91CF911F9161
:101C90000F91FF90EF90DF90CF90BF90AF909F900B
:101CA0007F906F905F904F900895EF92FF920F9307
:101CB0001F937B018C018091B7009091B800A09197
:101CC000B900B091BA008E159F05A007B10791F039
:101CD0000E94110CE092B700F092B8000093B90096
:101CE0001093BA004091AF005091B000C801B70105
:101CF0000E946C091F910F91FF90EF900895FA01D7
:101D00006083718382839383158214820E94800A88
:101D10000E94550E8091AF009091B0000895EF920F
:101D2000FF920F931F937B018C018091B3009091E0
:101D3000B400A091B500B091B6008E159F05A00724
:101D4000B10791F00E94920C4091B1005091B20005
:101D5000C801B7010E946C09E092B300F092B40090
:101D60000093B5001093B6001F910F91FF90EF9074
:101D70000895AF92BF92CF92DF92EF92FF920F93AE
:101D80001F937B018C0159016A010E94D30A0E94B2
:101D90008F0E8091C50082FF26C0F701EF77F070AB
:101DA000EE0FFF1FEE0FFF1F8091B1009091B20068
:101DB000E80FF91F80819181A281B38180709070BA
:101DC000A070B07F2FEF3FEF4FEF5FE0A222B32272
:101DD000C422D5228A299B29AC29BD2980839183DD
:101DE000A283B3830CC0F701F070EE0FFF1F809148
:101DF000B1009091B200E80FF91FB182A0828091EA
:101E0000C50080620E94780A1F910F91FF90EF90A9
:101E1000DF90CF90BF90AF900895AF92BF92CF92D6
:101E2000DF92EF92FF920F931F939B01AC01809181
:101E3000C50082FF73C0220F331F441F551FA32EFE
:101E4000B42EC52EDD248601750160915F05709169
:101E5000600580916105909162056E0D7F1D801F68
:101E6000911F0E948F0E8091C50082FF36C0E091C5
:101E7000B100F091B20060E070E080819181A281B8
:101E8000B381BF700097A105B10509F44CC06F5F25
:101E90007F4F34966038710581F70894E11CF11C7E
:101EA000011D111D8091670590916805A09169053C
:101EB000B0916A05E816F9060A071B0718F0EE2428
:101EC000FF248701AE14BF04C006D10609F0BDCFC0
:101ED00020E030E040E050E049C0E091B100F091F6
:101EE000B20060E070E080819181892B59F06F5FD2
:101EF0007F4F329681E06030780779F2808191815E
:101F0000892BA9F79B0144275527B02FAF2D9E2D74
:101F10008827280F391F4A1F5B1F28C0A32EB42E05
:101F2000C52EDD2490CF9B0144275527EE0CFF1CC6
:101F3000001F111FEE0CFF1C001F111FEE0CFF1CD9
:101F4000001F111FEE0CFF1C001F111FEE0CFF1CC9
:101F5000001F111FEE0CFF1C001F111FEE0CFF1CB9
:101F6000001F111F2E0D3F1D401F511FCA01B90137
:101F70001F910F91FF90EF90DF90CF90BF90AF90A7
:101F80000895EF92FF920F931F937B018C010E94A3
:101F9000D30A0E948F0E8091C50082FF1BC0F701FB
:101FA000EF77F070EE0FFF1FEE0FFF1F8091B10073
:101FB0009091B200E80FF91F608171818281938155
:101FC0009F70683F2FEF72072FEF82072FE0920775
:101FD000E8F018C0F701F070EE0FFF1F8091B1001C
:101FE0009091B200E80FF91F808191819C01B901A5
:101FF00088279927683F3FEF730730E0830730E079
:10200000930720F060E070E080E090E01F910F9176
:10201000FF90EF9008955F926F927F928F929F92C0
:10202000AF92BF92CF92DF92EF92FF920F931F93E6
:10203000CF93DF93582E8091C50083FF9FC080917E
:10204000570590915805A0915905B0915A05EC019A
:10205000D1709C01AD012F5F3F4F4F4F5F4F2093D9
:102060005705309358054093590550935A05213030
:1020700031054105510511F02097B1F160915305EB
:102080007091540580915505909156050E94550E0A
:102090008091AF009091B000C80FD91F58828091F5
:1020A000C50080650E94780A209157053091580537
:1020B0004091590550915A0580914F0590915005D6
:1020C000A0915105B091520582179307A407B50757
:1020D00040F420934F0530935005409351055093A1
:1020E000520581E090E0A6C080914F059091500587
:1020F000A0915105B0915205281739074A075B078F
:1021000008F43FC0E0905305F09054050091550548
:1021100010915605370148010894611C711C811CFF
:10212000911CC401B3010E94B80A5B016C01C80193
:10213000B7010E94B80A6A157B058C059D0599F4C4
:102140006092530570925405809255059092560501
:1021500060915305709154058091550590915605F5
:102160000E94700C8BCFC601B5010E940D0F5B0160
:102170006C016115710581059105C9F580E090E05C
:1021800059C0E0905305F090540500915505109109
:102190005605C801B7010E94B80A3B014C0157011E
:1021A00068010894A11CB11CC11CD11CC601B50159
:1021B0000E94B80A661677068806990649F4A09226
:1021C0005305B0925405C0925505D092560556CF8E
:1021D000C401B3010E94C10F0E94800A609353059D
:1021E00070935405809355059093560547CF6091A1
:1021F00053057091540580915505909156050E94A4
:10220000B80AA60195010E94B90E2FEF3FEF4FEFDC
:102210005FEFC601B5010E94B90EC601B5010E946B
:10222000800A6093530570935405809355059093ED
:1022300056058ECFDF91CF911F910F91FF90EF90B8
:10224000DF90CF90BF90AF909F908F907F906F90D6
:102250005F900895AF92BF92CF92DF92EF92FF927C
:102260000F931F93CF93DF930E94130B882371F575
:102270008091570590915805A0915905B0915A0544
:10228000EC01D1700196A11DB11D8093570590936B
:102290005805A0935905B0935A050197A105B105BA
:1022A00011F02097B1F06091530570915405809121
:1022B0005505909156050E94550E8091AF00909162
:1022C000B000C80FD91F8881992737C080E090E0FF
:1022D00034C0E0905305F0905405009155051091DD
:1022E0005605C801B7010E94B80A5B016C01089449
:1022F000E11CF11C011D111DC801B7010E94B80AA3
:10230000A616B706C806D90649F4E0925305F0921E
:1023100054050093550510935605C5CFC601B50168
:102320000E94C10F0E94800A609353057093540568
:102330008093550590935605B6CFDF91CF911F91AD
:102340000F91FF90EF90DF90CF90BF90AF900895E6
:102350006F927F928F929F92AF92BF92CF92DF92B5
:10236000EF92FF920F931F93CF93DF937B018C012A
:102370008091C50083FF08C0413009F47EC0413020
:1023800030F0423009F494C080E090E0A6C0A8018B
:102390009701E0925705F092580500935905109364
:1023A0005A058091470590914805AA27BB276C01E3
:1023B000BB24AA2480914D0590914E05AA27BB27E6
:1023C000A80EB91ECA1EDB1E39014A0121153105AE
:1023D0004105510551F0DA01C9019170A070B0704A
:1023E0000097A105B10509F45DC0C0912C05D091FD
:1023F0002D059E01322F2227330F44275527C40174
:10240000B3010E949B2479018A0121153105410500
:10241000510581F0C601B5010E94C10F5B016C013D
:102420000894E108F10801091109E114F10401051A
:10243000110581F709E096948794779467940A953B
:10244000D1F79E0144275527C401B3010E949B2464
:102450007B018C01C601B5010E94800AE60EF71EC1
:10246000081F191FE0925305F0925405009355057B
:102470001093560581E090E030C0209157053091CF
:1024800058054091590550915A052E0D3F1D401F8A
:10249000511F209357053093580540935905509389
:1024A0005A057FCF089461087108810891089DCF73
:1024B00020914F05309150054091510550915205A2
:1024C0002E193F09400B510B2093570530935805A7
:1024D0004093590550935A0564CFDF91CF911F91D6
:1024E0000F91FF90EF90DF90CF90BF90AF909F90B3
:1024F0008F907F906F900895DF92EF92FF920F93ED
:102500001F93CF93DF93EC018D818F5F8D8380319B
:10251000E0F11D82DC80D394DC828091C50082FDD5
:102520002FC0E880F9800A811B81E114F1040105C4
:10253000110589F12D2D332780912C0590912D05C2
:102540002817390708F044C0C801B7010E94800A63
:102550006D0D711D811D911D0E94550E8D81282FBD
:102560003327220F331F22953295307F3227207F69
:1025700032278091AF009091B000280F391F3AC0E8
:10258000E880F9800A811B81D5CFDC80E880F98062
:102590000A811B81D9CF8091630590916405A09138
:1025A0006505B09166058D0D911DA11DB11D209190
:1025B0005B0530915C0540915D0550915E05821789
:1025C0009307A407B50708F4BFCF20E030E012C09E
:1025D0001C82C801B7010E94C10F7B018C01688376
:1025E00079838A839B83611571058105910569F360
:1025F000DC80AACFC901DF91CF911F910F91FF908D
:10260000EF90DF9008950F931F93CF93DF93CDB793
:10261000DEB726970FB6F894DEBF0FBECDBF8E0192
:102620000F5F1F4FA8010E947F0EFC01892B69F0EC
:1026300080818E3221F0882341F0853E49F4C80123
:102640000E947C12FC01892B99F781E090E002C086
:1026500080E090E026960FB6F894DEBF0FBECDBFA7
:10266000DF91CF911F910F910895AF92BF92CF92BA
:10267000DF92EF92FF920F931F93CF93DF93CDB72B
:10268000DEB763970FB6F894DEBF0FBECDBF5C0117
:10269000E7E0CE2ED12CCC0EDD1E4CE050E0C60182
:1026A0000E944C241B8AC6010E94840B609128055D
:1026B0007091290580912A0590912B057E0108943F
:1026C000E11CF11CA7010E947F0E8C01892BA9F44B
:1026D00022C0853E61F0F80183858F3041F04BE0E8
:1026E00050E0B601C8010E943E24892B69F0C70161
:1026F0000E947C128C01892B71F0F8018081882363
:1027000041F700E010E007C0D501F80180E2019038
:102710000D928150E1F7C80163960FB6F894DEBFC1
:102720000FBECDBFDF91CF911F910F91FF90EF9022
:10273000DF90CF90BF90AF9008950F931F93CF93EA
:10274000DF93CDB7DEB7A7970FB6F894DEBF0FBE05
:10275000CDBF8091C500992783FF02C084FD07C0CB
:102760000E94920C0E94110C81E090E0B1C063E3E2
:1027700075E0CE0108960E9435138C01892B09F46F
:10278000A1C080914F0590915005A0915105B09145
:102790005205F801848F958FA68FB78FCE010196D1
:1027A0000E94E9184E815527440F551F42955295B6
:1027B000507F5427407F54278D819927982F882751
:1027C000990F990F990F2F812695820F911D480F10
:1027D000591F2A813327220F331F22953295307FCC
:1027E0003227207F32278B819C818C5B9740982FEA
:1027F0008827990F6981860F911D280F391FF801CD
:10280000468B452F5527478B208F832F9927818F04
:10281000228B838B8091C50080640E94780A80910E
:10282000C50082FD04C08F7E0E94780A99CF609116
:102830006B0570916C0580916D0590916E050E94FD
:10284000550EE091AF00F091B000E851FE4F8FEFD0
:102850008083E091AF00F091B000E751FE4F80839C
:10286000E091AF00F091B000E651FE4F8083E0911F
:10287000AF00F091B000E551FE4F8083E091AF00D2
:10288000F091B000E451FE4F8083E091AF00F091F1
:10289000B000E351FE4F8083E091AF00F091B000B3
:1028A000E251FE4F8083E091AF00F091B000E15122
:1028B000FE4F80838091C50080640E94780A8091D9
:1028C000C500B1CF0E94920C0E94110C80E090E0F4
:1028D000A7960FB6F894DEBF0FBECDBFDF91CF91A4
:1028E0001F910F9108950E949D138091C500877FCD
:1028F0000E94780A81E090E008950F931F938C0165
:102900000E949D13B80183E395E00E943513892B43
:10291000C9F10091C50002FF2CC06091470570917C
:10292000480588279927CB017727662720914D05F1
:1029300030914E0544275527620F731F841F951F42
:102940000E94800A1092570510925805109259055E
:1029500010925A0560935305709354058093550562
:1029600090935605802F88600E94780A81E090E05D
:102970000BC060914D0570914E05882799270E94E4
:10298000800AE0CF80E090E01F910F9108956F9250
:102990007F928F929F92AF92BF92CF92DF92EF92EF
:1029A000FF920F931F93CF93DF93CDB7DEB7A0971E
:1029B0000FB6F894DEBF0FBECDBFBC01CE010196AD
:1029C0000E9435138C01009709F445C06090B70050
:1029D0007090B8008090B9009090BA00FC01848992
:1029E0009589AA27BB276C01BB24AA24828D938DCD
:1029F000AA27BB27A80EB91ECA1EDB1E83858031FD
:102A000021F1C401B3010E94550E85EEF8018083C7
:102A10008091C50080640E94780AC601B5010E94B9
:102A2000C10F7B018C0120E030E040E050E0C601A6
:102A3000B5010E94B90E57016801E114F1040105C6
:102A4000110559F781E090E008C0C601B5010E9468
:102A500003138823B1F680E090E0A0960FB6F894B7
:102A6000DEBF0FBECDBFDF91CF911F910F91FF90C1
:102A7000EF90DF90CF90BF90AF909F908F907F901E
:102A80006F900895CF92DF92EF92FF920F931F9372
:102A9000CF93DF93CDB7DEB7AD970FB6F894DEBF17
:102AA0000FBECDBF6C018B013EE0E32EF12CEC0E8E
:102AB000FD1EC7010E943513892B19F080E090E0BC
:102AC00022C0B601C7010E9435137C01892BB1F3E6
:102AD0004CE050E0B8018E010F5F1F4FC8010E940B
:102AE0004C241D86C8010E94840BF701D8018BE09D
:102AF0000D9001928150E1F78091C50080640E94A1
:102B0000780A81E090E0AD960FB6F894DEBF0FBE74
:102B1000CDBFDF91CF911F910F91FF90EF90DF908C
:102B2000CF900895CF93DF93CDB7DEB7A0970FB6C0
:102B3000F894DEBF0FBECDBFFC0180818F32E9F17A
:102B4000BF01CE0101960E943513892B99F18C8526
:102B500084FF30C08B8D9C8D9C01442755278D8927
:102B60009E89AA27BB27DC0199278827280F391FB0
:102B70004A1F5B1F209328053093290540932A059F
:102B800050932B058091C50082FF2AC02115310585
:102B90004105510529F582E090E0A0E0B0E0809386
:102BA000280590932905A0932A05B0932B0581E071
:102BB00090E018C080E090E015C080916F05909182
:102BC0007005A0917105B0917205809328059093CE
:102BD0002905A0932A05B0932B0581E090E002C05F
:102BE00081E090E0A0960FB6F894DEBF0FBECDBF97
:102BF000DF91CF910895CF92DF92EF92FF920F93E2
:102C00001F93CF93DF93CDB7DEB726970FB6F89417
:102C1000DEBF0FBECDBF7B018C016E010894C11CCD
:102C2000D11CA6010E947F0EFC01892B71F411C0FA
:102C3000882309F441C0E980FA800B811C81C60118
:102C40000E947C12FC01892B21F08081853E81F756
:102C500033C08091C50082FD05C0E114F104010577
:102C6000110559F0C801B7010E940D0F9B01AC017D
:102C7000611571058105910519F4E0E0F0E01CC0D3
:102C800069837A838B839C83C801B7010E94B90E44
:102C900069817A818B819C812FEF3FEF4FEF5FEF4E
:102CA0000E94B90E69817A818B819C810E942B0CD4
:102CB000E091AF00F091B000CF0126960FB6F894E6
:102CC000DEBF0FBECDBFDF91CF911F910F91FF905F
:102CD000EF90DF90CF9008956F927F928F929F92A6
:102CE000AF92BF92CF92DF92EF92FF920F931F931A
:102CF000CF93DF93CDB7DEB7E4970FB6F894DEBF7E
:102D00000FBECDBF6C01BC01CE0145960E943513AC
:102D1000892B19F080E090E095C0609128057091B2
:102D2000290580912A0590912B050E94FB157C01B5
:102D3000892B81F3609128057091290580912A05DE
:102D400090912B050E940D0F3B014C0161157105FF
:102D500081059105F9F28E01085F1F4F4CE050E0AC
:102D6000B601C8010E944C241C8AC8010E94840B31
:102D7000CE0101960E94E9188E81A82EBB24AA0CD0
:102D8000BB1CA294B29450EFB522BA24A522BA2457
:102D90008D819927982F8827990F990F990F2F8147
:102DA0002695820F911DA80EB91E8A81682F77275C
:102DB000660F771F62957295707F7627607F762702
:102DC0008B819C818C5B9740982F8827990F298154
:102DD000820F911D680F791FF701D8018BE00D90CC
:102DE00001928150E1F780E2F7018387148615860E
:102DF000A6864B2D55274787608B272F3327218B9E
:102E0000628B238BC401AA27BB27958B848BA68A50
:102E1000478B608F218F738E628E148E158E168E67
:102E2000178E8091C50080640E94780A2FEF3FEFD3
:102E30004FEF5FEFC401B3010E94B90EC6010E94BB
:102E40007D149927E4960FB6F894DEBF0FBECDBF70
:102E5000DF91CF911F910F91FF90EF90DF90CF9076
:102E6000BF90AF909F908F907F906F9008954F92FA
:102E70005F926F927F928F929F92AF92BF92CF920A
:102E8000DF92EF92FF920F931F93CF93DF93CDB713
:102E9000DEB7E4970FB6F894DEBF0FBECDBF7C015E
:102EA000BC01CE0145960E943513892B19F080E0B4
:102EB00090E0F8C0609128057091290580912A055D
:102EC00090912B050E94FB156C01892B81F3609179
:102ED00028057091290580912A0590912B050E9463
:102EE0000D0F4B015C016115710581059105F9F22A
:102EF0008E01085F1F4F4CE050E0B701C8010E94EF
:102F00004C241C8AC8010E94840BCE0101960E94A9
:102F1000E9188E81E82EFF24EE0CFF1CE294F29457
:102F200050EFF522FE24E522FE248D819927982F6B
:102F30008827990F990F990F2F812695820F911D40
:102F4000E80EF91E8A81682F7727660F771F629532
:102F50007295707F7627607F76278B819C818C5B52
:102F60009740982F8827990F2981820F911D680F0C
:102F7000791FF601D8018BE00D9001928150E1F7A5
:102F800080E1F6018387148615866E2CE6864F2D28
:102F90005527742E4787162F608B272F3327022F34
:102FA000218B628B238BC501AA27BB272C01958B14
:102FB000848BE68A478B608F218F7401938E828E7B
:102FC000148E158E168E178E8091C50080640E9417
:102FD000780AC501B4010E942B0C4091AF005091BA
:102FE000B000DA0127E930E08BE0F90101909F01A0
:102FF0000D928150D1F780E1FA01838714861586FE
:1030000066867786108B018B128B038B558A448AD8
:10301000668A778A108F018FF38EE28E148E158E5A
:10302000168E178E9A01205E3F4FF901A3EAB0E099
:103030008BE00D9001928150E1F780E1F9018387E7
:103040001486158666867786108B018B128B038B10
:103050008091280590912905A0912A05B0912B0512
:10306000CD01AA27BB27958B848B668A778A108F20
:10307000018F8091280590912905938F828F148E5E
:10308000158E168E178E8091C50080640E94780A76
:103090002FEF3FEF4FEF5FEFC501B4010E94B90E74
:1030A00081E090E0E4960FB6F894DEBF0FBECDBF8E
:1030B000DF91CF911F910F91FF90EF90DF90CF9014
:1030C000BF90AF909F908F907F906F905F904F9048
:1030D00008950E946C09992708959198899A84E12E
:1030E00090E00E946802919A80E00E94780A8FEF37
:1030F0009FEFAFEFBFEF8093B3009093B400A09326
:10310000B500B093B6008093B7009093B800A09339
:10311000B900B093BA004091AF005091B00060E0A8
:1031200070E080E090E00E946C09E091AF00F091C7
:10313000B000E250FE4F8081EE5FF140853519F01E
:1031400080E090E00895E150FE4F8081EF5FF14014
:103150008A3AB1F7E254FE4F80818068803859F096
:1031600060E070E080E090E00E94A70D8823C9F045
:1031700081E090E0089584818D30D8F48B30E0F4C4
:10318000843011F0863061F78091C50082608093B1
:10319000C50060857185828593850E94DD0C992725
:1031A000089560E070E080E090E00E94DD0C9927D7
:1031B00008958E30A9F6E8CF8091C5008260809393
:1031C000C50060857185828593850E94A70D99272A
:1031D0000895FC0181E08083818387ED97E09383EC
:1031E000828381E184838EE18583168208958091B4
:1031F0007505992780FF02C081FD03C081E090E042
:103200000895969587959695879581709070089505
:103210008091750581708093750581E090E0089537
:10322000809175059927089580E090E008950E94A7
:10323000010B60507B4A8240904030F081E08093E7
:10324000750581E090E008951092750580E090E0AA
:103250000895CF92DF92EF92FF920F931F93582F12
:10326000C62ED82EDA94862F9927DD2079F020E01B
:1032700030E041E0E22FFF27EF55FE4FE4918E0F43
:10328000911D2F5F3F4F4F5F5417A1F7AA27BB2710
:10329000EE24F82E092F1A2F0E94010BE616F706CE
:1032A0000807190718F01092750514C040E0C8010E
:1032B000B7010E94A8110E942A11809374050E94F0
:1032C0002A1180937805D0927705C092730582E029
:1032D000809376051F910F91FF90EF90DF90CF9034
:1032E00008958091750580FF089560E082E10E9455
:1032F000291941E06EE870E080E090E00E94A8119A
:1033000081E08093750508950F931F93CF93DF930A
:10331000AC0180917505282F332720FF21C023FFA2
:103320001FC024FD1DC0EA018A01025E1F4F0E94DA
:103330002A118993809176058F5F80937605C01757
:10334000D107A9F78823B1F480917405882359F433
:103350008091750580618093750581E090E01BC0C8
:1033600080E090E018C0609178050E94291981E002
:1033700090E011C00E942A11182F0E942A11982F44
:10338000809176058E5F80937605112311F49F3F1F
:10339000F9F281E090E0DF91CF911F910F910895B4
:1033A0008091750580FD03C080E090E0089561E0A4
:1033B00082E10E94291989E08093750581E090E0FF
:1033C00008958F929F92AF92BF92CF92DF92EF9229
:1033D000FF920F931F93CF93DF93CDB7DEB7ED9797
:1033E0000FB6F894DEBF0FBECDBF6C01809175059E
:1033F00080FD11C08E01015E1F4F4AE050E069EE72
:1034000071E0C8010E941C24A8016AE080E090E0FD
:10341000F6010995C6C00E94711982E18F8F82E280
:1034200088A302E07FE1E72EF12CEC0EFD1E0E9446
:103430002A11803A09F4A4C0023109F499C0F701B5
:10344000E00FF11D80830F5F093188F3A70169E167
:1034500080E090E0F601099543E050E060E270E022
:10346000C7010E94252482E28AA30E94D0198E01FE
:103470000F5F1F4F63E2862E912C8C0E9D1E55E32D
:10348000A52EB12CAC0EBD1EC8010E948419882344
:1034900009F458C08A818823B9F34AE150E060E218
:1034A00070E0C4010E94252484E090E09E012C5F1E
:1034B0003F4F482FDC01F9018081803A71F0F7011C
:1034C000EA0FFB1F80834F5FCD0101962F5F3F4FB7
:1034D0008431910571F7A42FBB27AE0DBF1D82E289
:1034E0008C9389818770863008F085E063E0869F41
:1034F000B001112467537E4F43E050E0C5010E94A4
:103500001C24998196FF02C08CE388AF97FD02C00E
:103510008AE289AF2D8D8E8D9927982F8827820F6B
:10352000911DF3E0883E9F0768F143E050E04E0DA7
:103530005F1D6BE1F6010995C8010E94841988237B
:1035400009F0A8CF4CE050E06CED71E0C7010E949B
:103550001C244DE050E060E270E0CE018B960E94AA
:103560002524A70169E180E090E0F601099519C0E2
:1035700082E289AB03E10E942A11803A09F05CCF14
:1035800080E25ACF8436910530F440E08A309105CC
:1035900028F45527CCCF42E050E0C9CF41E0552771
:1035A000C6CFED960FB6F894DEBF0FBECDBFDF914C
:1035B000CF911F910F91FF90EF90DF90CF90BF9030
:1035C000AF909F908F900895CF92DF92EF92FF92ED
:1035D0000F931F93CF93DF93CDB7DEB76E970FB6E0
:1035E000F894DEBF0FBECDBF6C0160E170E00E94B9
:1035F0005B24082F0E94D01910E07E010894E11C82
:10360000F11CC7010E948419882309F446C08981EE
:1036100087708150823038F010E0C7010E94841911
:103620008823A9F73AC0002371F111E090E005C0AA
:103630009F5F0917B9F0112321F3A92FBB27F601CA
:10364000EA0FFB1F20812F3399F32A32C9F010E0D3
:10365000AE0DBF1DFD018381281751F711E09F5F5B
:10366000091749F7112369F2003168F0112349F273
:103670006B818A810E94291983E0809375050DC0B2
:103680000917A1F7F1CF10E0F701E00FF11D8381D9
:10369000803A09F0B6CF11E0EBCF812F99276E96D3
:1036A0000FB6F894DEBF0FBECDBFDF91CF911F9153
:1036B0000F91FF90EF90DF90CF9008951F930E949D
:1036C000F718882319F080E090E01FC00E942A11AB
:1036D000182F809176058F3F31F08F5F80937605AC
:1036E000812F992712C080917405882341F480911D
:1036F0007505846080937505812F992706C06091B8
:1037000078050E942919812F99271F91089580918A
:103710008105992780FF02C081FD03C081E090E010
:1037200008959695879596958795817090700895E0
:1037300080918105992708958091810581708093FA
:10374000810581E090E008958091810580FD03C0AE
:1037500080E090E0089540E060E470E080E090E078
:103760000E94A81189E08093810510927A05109239
:10377000790580917B0590917C05892B31F489E155
:103780008093810581E090E0089581E090E00895C4
:103790008091810580FF089540E068E270E080E05C
:1037A00090E00E94A81181E0809381050895109215
:1037B00081050E94010B603471058105910518F4A3
:1037C00080E090E0089540E060E070E080E090E00C
:1037D0000E94A8110E942A11833491F70E942A1195
:1037E000863371F70E942A11843351F740E062E278
:1037F00070E080E090E00E94A8110E942A119927B1
:1038000090937C0580937B0540E063E270E080E06C
:1038100090E00E94A8110E942A119927982F8827CA
:1038200020917B0530917C05282B392B30937C052A
:1038300020937B0581E08093810581E090E00895ED
:103840000F931F93CF93DF93AC0180918105282FB5
:10385000332720FF21C023FF1FC024FD1DC0EA0124
:103860008A01005E1F4F0E942A118993C017D10759
:10387000D1F78091790590917A05019690937A0518
:103880008093790520917B0530917C058217930701
:1038900031F081E090E00AC080E090E007C08091C4
:1038A000810580618093810581E090E0DF91CF9177
:1038B0001F910F9108950E94871B882399F480918E
:1038C0007D0590917E052FEF8E3F920721F18F5F4E
:1038D0009F4F59F48091830510927E0510927D05CB
:1038E0009927089580E090E008950E942A11482FBA
:1038F00080917D0590917E05019690937E05809341
:103900007D0520917F05309180058217930771F026
:10391000842F99270895209182058FEF9FEF909330
:103920007E0580937D05822F9927089580918105DA
:10393000846080938105842F99270895CF92DF9228
:10394000EF92FF920F931F93CF93DF93CDB7DEB724
:10395000E6970FB6F894DEBF0FBECDBF6C010E9494
:10396000C81B82E1898382E28A838E010D5F1F4F2B
:1039700046E1E42EF12CEC0EFD1E06C0F801819309
:103980008F01EE15FF0559F00E942A11803AB1F718
:1039900080E2F80181938F01EE15FF05A9F712E28D
:1039A0001B8B7E010894E11CF11CA70166E180E0FD
:1039B00090E0F601099580E289838A831B831C8B42
:1039C0000E94A41B8E01095E1F4FC8010E94201C8B
:1039D0008823D1F08F898823C1F3888D8823A9F3A8
:1039E000DE011496FE01B79680E101900D928150A0
:1039F000E1F7A70164E180E090E0F6010995C801D4
:103A00000E94201C882331F749E050E064EF71E008
:103A1000C7010E941C24A70169E080E090E0F60144
:103A20000995E6960FB6F894DEBF0FBECDBFDF91C5
:103A3000CF911F910F91FF90EF90DF90CF9008955D
:103A4000CF92DF92EF92FF920F931F93CF93DF936A
:103A5000CDB7DEB7A0970FB6F894DEBF0FBECDBFCF
:103A60008C01FC0101900020E9F73197FE2EF81A35
:103A700080E18F1510F490E1F92E0E94A41BEE2432
:103A80006E010894C11CD11CC6010E94201C882311
:103A900009F46DC08981882309F459C08A8188237B
:103AA00009F455C0FF2009F457C081E0E82E90E0EA
:103AB00005C09F5FF916C9F0EE2031F3A92FBB278F
:103AC000F801EA0FFB1F20812F3399F32A3209F402
:103AD00040C0EE24AC0DBD1DFD018089281749F7BB
:103AE000B1E0EB2E9F5FF91639F7EE2069F2FFE0A7
:103AF000FF1590F5EE2041F26B81609382054C81B9
:103B0000409383058EEF9FEF90937E0580937D0514
:103B10002D8133278E819927982F8827282B392BA1
:103B200077275527542F4427642B752B261B370BDB
:103B30003093800520937F0569857A858B859C85E8
:103B400040E00E94A81183E08093810510C0EE241C
:103B50009BCFF91679F6CBCFEE24F601EF0DF11DD0
:103B60008089803209F090CFA1E0EA2EC5CF8E2D5A
:103B70009927A0960FB6F894DEBF0FBECDBFDF9198
:103B8000CF911F910F91FF90EF90DF90CF9008950C
:103B9000809184058E7F809384050E94731481E058
:103BA00090E00895982F8091840580FD03C080E007
:103BB00090E00895892F0E940B1099270895809115
:103BC000840580FD03C081E090E008950E94130BFE
:103BD000992708958091840580FD03C080E090E0DE
:103BE00008950E942A1199270895CF92DF92EF92AB
:103BF000FF920F931F93CF93DF937C016B010E9481
:103C0000130B882319F080E090E02DC00E942A1148
:103C1000082F0E942A118A33B1F7E70110E00E94B1
:103C20002A11E114F10409F088831F5F21961C30EA
:103C3000B1F70E942A118A3331F7E60110E00E94A1
:103C40002A11C114D10409F088831F5F2196103115
:103C5000B1F70E942A118D30B1F60E942A118A30E4
:103C600091F6802F9927DF91CF911F910F91FF90AF
:103C7000EF90DF90CF900895EF92FF921F93CF9334
:103C8000DF93EC017C0110E00E942A11E114F104A1
:103C900009F088831F5F21961031B1F70E942A1125
:103CA0008D3019F080E090E00AC00E942A1190E067
:103CB0008A3009F091E081E09827892F9927DF91D8
:103CC000CF911F91FF90EF900895AF92BF92CF9246
:103CD000DF92EF92FF920F931F93CF93DF93CDB7B5
:103CE000DEB76B970FB6F894DEBF0FBECDBF7C0179
:103CF0001092840585E895E00E947D14882309F4DC
:103D00004DC082E1898302E20A83CE0103960E94BC
:103D10003C1E182F0B8B44E050E065E172E0CE01B1
:103D200044960E941C241123C9F15E010894A11C31
:103D3000B11CA50167E180E090E0F701099580E200
:103D400089838A830B830C8B8D8B8E010C5F1F4FB5
:103D500086E1C82ED12CCC0EDD1E0E94130B8823C9
:103D6000D1F4B80180E090E00E94F51D803539F172
:103D7000843499F761E172E043E050E0C6010E94AB
:103D80001C24A50168E180E090E0F70109950E94FC
:103D9000130B882331F30E94731414C04EE050E0DB
:103DA0006EEF71E08E010F5F1F4FC8010E941C244F
:103DB000A8016EE080E090E0F701099503C06DE096
:103DC00072E0DACF6B960FB6F894DEBF0FBECDBFB0
:103DD000DF91CF911F910F91FF90EF90DF90CF90E7
:103DE000BF90AF900895AF92BF92CF92DF92EF92C3
:103DF000FF920F931F93CF93DF93CDB7DEB72D972D
:103E00000FB6F894DEBF0FBECDBF5C0110928405E3
:103E100048E050E0BC016E010894C11CD11CC601F1
:103E20000E944C2468E070E0C6010E945B24883048
:103E300008F47AC045E050E060E272E0CE010996F5
:103E40000E941C24EE24FF2410C00894E11CF11CE5
:103E500085E6E816F104A9F0812F6AE00E948F241C
:103E6000191B105D1F83905D98871E2DC6010E944F
:103E70007D14882351F785E895E00E947D148823FE
:103E800019F480E090E05CC080E090E00E943C1E6D
:103E90008823B9F342E060E070E080E090E00E94A7
:103EA000A81180E50E940B108AE30E940B10760196
:103EB0008E01035F1F4FF70181917F010E940B105C
:103EC000E016F106C1F78AE30E940B10F50110819C
:103ED000750100E00BC0812F0E940B10F7011181CA
:103EE0000F5F0894E11CF11C003159F0112399F780
:103EF00080E20E940B100F5F0894E11CF11C00315E
:103F0000A9F78DE00E940B108AE00E940B100E941E
:103F10007314C6010E946C168091840581608093A1
:103F2000840581E090E00CC0992748E050E0481BF0
:103F3000590B60E270E08C0D9D1D0E9425247ACF04
:103F40002D960FB6F894DEBF0FBECDBFDF91CF9197
:103F50001F910F91FF90EF90DF90CF90BF90AF90A7
:103F60000895BF92CF92DF92EF92FF920F931F932B
:103F7000CF93DF936C017B01EA01B22E222379F00B
:103F800085E895E00E947D14882331F080E090E080
:103F90000E943C1E882381F480E090E067C040E0EE
:103FA00060E070E080E090E00E94A81180E090E086
:103FB0000E943C1E882381F360E170E0CE010E94E4
:103FC0005B24182F882319F409C0115039F0FE0121
:103FD000E10FF11D319780818032B9F300E00E943A
:103FE000130B8823A1F5B701C6010E94F51D80358A
:103FF000A9F7F7013F9620E18081803221F421501A
:1040000031972223C9F71123F1F090E001E005C0B8
:104010009F5F9117B1F0002311F3A92FBB27FE0179
:10402000EA0FFB1FE081EF3399F3EA32A9F000E0D9
:10403000AE0DBF1D8C91E81759F701E09F5F9117F6
:1040400051F7002361F200E0211749F601E0BB209F
:1040500051F4802F99270AC09117A9F3002309F47E
:10406000BECFBB20B1F30E947314F3CFDF91CF9189
:104070001F910F91FF90EF90DF90CF90BF90089528
:10408000EF92FF920F931F93CF93DF93CDB7DEB7DD
:104090006C970FB6F894DEBF0FBECDBF7C011092B7
:1040A000840521E0AC01BE01635F7F4F8E010F5F8D
:1040B0001F4FC8010E94B11F882361F0C8010E94F0
:1040C000C714C8010E946C1680918405816080939A
:1040D000840505C0C7010E94F31E809184059927BD
:1040E000817090706C960FB6F894DEBF0FBECDBF96
:1040F000DF91CF911F910F91FF90EF9008950F9353
:104100001F93CF93DF93CDB7DEB76C970FB6F894BC
:10411000DEBF0FBECDBF1092840521E0AC01BE0111
:10412000635F7F4F8E010F5F1F4FC8010E94B11F59
:10413000882319F4809184050AC0C8010E947D1467
:104140008823C1F380918405816080938405992739
:10415000817090706C960FB6F894DEBF0FBECDBF25
:10416000DF91CF911F910F910895CF92DF92EF923F
:10417000FF920F931F93CF93DF93CDB7DEB7609776
:104180000FB6F894DEBF0FBECDBF8C016B018091DE
:1041900084058E7F8093840585E895E00E947D14D8
:1041A000882319F400E010E035C020E0A801BE012A
:1041B0006F5F7F4F80E090E00E94B11F882329F459
:1041C00000E010E00E94731425C041E06EEE7FEF26
:1041D0008FEF9FEF0E94A811F601F0808601EE2478
:1041E0000BC08F2D0E940B10F801F180E3940F5F3C
:1041F0001F4FF0E1EF1659F0FF2099F780E20E947F
:104200000B10E3940F5F1F4FF0E1EF16A9F701E0E9
:1042100010E0D8CFC80160960FB6F894DEBF0FBE8D
:10422000CDBFDF91CF911F910F91FF90EF90DF9065
:10423000CF900895BF92CF92DF92EF92FF920F93AB
:104240001F93CF93DF93CDB7DEB76C970FB6F8947B
:10425000DEBF0FBECDBF7C01809184058E7F809331
:10426000840585E895E00E947D14882361F1BB24D4
:104270002DE0C22ED12CCC0EDD1E8E010F5F1F4F04
:1042800015C041E06FED7FEF8FEF9FEF0E94A81107
:104290008DE20E940B100E947314C8010E94C71483
:1042A00085E895E00E947D1491E0B92E20E0A701F9
:1042B000B601C8010E94B11F882319F70E94731428
:1042C0008B2D992702C080E090E06C960FB6F89491
:1042D000DEBF0FBECDBFDF91CF911F910F91FF9039
:1042E000EF90DF90CF90BF900895CF92DF92EF9242
:1042F000FF920F931F93CF93DF93CDB7DEB72D9728
:104300000FB6F894DEBF0FBECDBF8C01809184053F
:104310008E7F8093840548E050E0B8016E010894D8
:10432000C11CD11CC6010E944C2468E070E0C6018B
:104330000E945B24883008F444C045E050E06AE104
:1043400072E0CE0109960E941C24C6010E947D14D1
:10435000882329F00E94731485E090E040C0C601D4
:104360000E946C168823C9F1F801F080EE240BC07E
:104370008F2D0E940B10F801F180E3940F5F1F4F07
:10438000F0E1EF1659F0FF2099F780E20E940B1040
:10439000E3940F5F1F4FF0E1EF16A9F78DE00E9445
:1043A0000B108AE00E940B100E947314A5E8B5E080
:1043B000F6018DE001900D928150E1F780E090E0F0
:1043C0000EC0992748E050E0481B590B60E270E0AE
:1043D0008C0D9D1D0E942524B0CF82E090E02D968B
:1043E0000FB6F894DEBF0FBECDBFDF91CF911F9106
:1043F0000F91FF90EF90DF90CF9008951F93CF9390
:10440000DF93FC0110816AE370E00E942C24009786
:10441000D1F0EC0121961335F1F0123529F01E345C
:10442000A9F083E090E01EC06DE370E0CE010E9431
:104430002C24FC01892B39F01192BE01CF010E947E
:10444000B520882369F080E090E00CC0CE010E9486
:104450007521992707C0CE010E941A21882399F758
:1044600084E090E0DF91CF911F9108951F93FC01AC
:1044700001900020E9F73197E81BF90B3D9718F000
:1044800080E090E010C0BC0185E895E00E943724F0
:104490001092840580E090E00E943C1E182F0E943C
:1044A0007314812F99271F91089591E0EAE9F5E0AF
:1044B000A2E9B5E02FEF9ABB1BBA2BBB1BBA8081D8
:1044C0008D9383B381932BBB1ABA990F85E0E23A9F
:1044D000F80789F708958091CE0099270895809173
:1044E000CE0081FD06C080FF089589E50E94580A2C
:1044F000089582E10E94580A8091CE00F4CF1F9364
:10450000182F80EF0E94580A812F0E94580A0E949B
:104510006F221F9108958091CE0081FD09C080FF18
:10452000089580EF0E94580A89E50E94580A08956C
:1045300080EF0E94580A82E10E94580A8091CE00C2
:10454000EECF4F925F926F927F928F929F92AF9237
:10455000BF92CF92DF92EF92FF920F931F93CF9370
:10456000DF930E9455225EE2852E52E0952E42E9AD
:10457000642E45E0742E3AE9432E35E0532E21E0B7
:10458000A22EF301B080F201E08098EFC92E9FEFD8
:10459000D92EC80CD91C0DC02230310509F45DC0DC
:1045A0000894C11CD11CC814D90409F406C1B694DE
:1045B000E694F601F4902B2D332721703070220FF2
:1045C000331F8E2D992781709070282B392B213025
:1045D000310511F7FDE3FF1609F48FC08CE4F816DE
:1045E00009F49CC09FEFF91609F4A3C0A0E0B0E065
:1045F000EBEBF0E0C6ECD0E007C0119631962196C7
:10460000A430B10509F460C08081F816B1F7888143
:10461000813099F7FD01E154FF4F1081AA53BF4F3C
:104620001C9217FD54C080EF0E94580A812F8F778B
:104630000E94580A123109F46BC0193509F0B0CF45
:104640008091CE008E7F8093CE000894C11CD11C37
:10465000C814D90409F0ABCFB0C0EDE3FE1609F4DD
:1046600079C0FCE4FF1609F482C08FEFF81609F454
:104670008BC0C0E0D0E00BEB10E006C021960F5FCE
:104680001F4FC430D10539F1F8018081F816B1F718
:104690000E946B22882391F3FE01E154FF4F1081A9
:1046A000CA53DF4FA88217FD19C0812F8F770E9450
:1046B000580A1231E1F0193509F072CF8091CE001D
:1046C00081608093CE006CCF1F2D17FFACCF80EEA2
:1046D0000E94580AA8CF1F2D17FFE7CF80EE0E9437
:1046E000580A812F8F770E94580A123121F7809142
:1046F000CE0082608093CE0053CF8091CA0081307B
:1047000009F074CF1092CA0082E50E947F2248CF40
:104710008091CE008D7F8093CE0042CF8091CD00DE
:10472000813009F063CF1092CD008BE50E947F228B
:1047300037CF8091CC00813099F180EF0E94580AE8
:104740008CE40E94580A80EF0E94580A82E10E947D
:10475000580A26CF0E946B22882309F48ACFA092A0
:10476000CA000E948B2282E50E94580A19CF0E943B
:104770006B22882309F47DCFA092CD000E948B226A
:104780008BE50E94580A0CCF0E946B22882371F09F
:10479000A092CC000E948B2284E50E94580A00CF90
:1047A0001092CC0084E50E947F22FACE82E10E9422
:1047B000580A8CE40E94580AF3CE0894611C711CBC
:1047C0000894411C511C88E090E0880E991E9AE9DB
:1047D000691695E0790609F0D4CEDF91CF911F914B
:1047E0000F91FF90EF90DF90CF90BF90AF909F9090
:1047F0008F907F906F905F904F9008950E94430A32
:10480000E2E9F5E0AAE9B5E08FEF81938D9395E0B9
:10481000EA39F907D1F71ABA14BA85BB0895FB0132
:10482000DC0104C08D910590801921F44150504065
:10483000C8F7881B990B0895FB01DC0102C00590A5
:104840000D9241505040D8F70895DC0101C06D939E
:1048500041505040E0F70895FC018191861721F006
:104860008823D9F7992708953197CF010895FB013F
:10487000DC0101900D920020E1F70895FB01DC01BD
:104880004150504030F08D910190801919F4002072
:10489000B9F7881B990B0895FB01DC01415050408A
:1048A00048F001900D920020C9F701C01D924150BF
:1048B0005040E0F70895FC016150704001900110F4
:1048C000D8F7809590958E0F9F1F0895DC016C910D
:1048D00061566A3108F0605E6F5B6D93C1F70895B1
:1048E000629FD001739FF001829FE00DF11D649FD4
:1048F000E00DF11D929FF00D839FF00D749FF00D60
:10490000659FF00D9927729FB00DE11DF91F639F00
:10491000B00DE11DF91FBD01CF0111240895991BB0
:1049200079E004C0991F961708F0961B881F7A95A6
:10493000C9F780950895A1E21A2EAA1BBB1BFD01A1
:104940000DC0AA1FBB1FEE1FFF1FA217B307E4076E
:10495000F50720F0A21BB30BE40BF50B661F771FC6
:10496000881F991F1A9469F76095709580959095A6
:0C4970009B01AC01BD01CF010895FFCFF9
:10497C0000CA9A3B00E1F5058096980040420F0072
:10498C00A086010010270000E8030000640000006E
:10499C000A000000010000002E2E00464154313662
:1049AC00004641543332002E20202020202020208D
:1049BC002020002E2E202020202020202020002807
:1049CC00012803FFFFFFFFFFFFFFFF1E363E46528D
:0449DC003D4645000F
:00000001FF
